Question link: http://acm.hdu.edu.cn/showproblem.php? PID = 1, 3132
Problem descriptionthe brave knights of Camelot are constantly exposed to French taunting while assaulting the castle occupied by the French. consequently, the taunting to which they are exposed varies with their distance from the castle during their assault, as well as variations in French taunting activity. we need to estimate the total amount of taunting that they are exposed to d
Portal: Windy and Mercury-Mercury Games 1Test instructions: On a chessboard composed of N*m, the K Knight is placed on the board of each knight (Xi,yi), indicating the first XI line, the Knight row if the current position is (x, y), a step can go to the position of(x-2,y-1)(x-2,y+1)(x-1,y-2)(x+1,y-2)Two people, each move a knight, at the same time can have more than one knight in the same lattice, who can not move who loses now given the initial chess face, ask the initiator whether there is a w
Http://poj.org/problem? Id = 3132
Question:
Given N and K, the number of N schemes is represented by exactly k different prime numbers.
Analysis:
N and K are both small. It's a backpack. You just need to select K items to fill up n.
1 #include
# Include # include using namespace STD; struct DNA {int A, C, G, T;} d [1005]; int main (INT argc, char * argv []) {int t, n, m, I, j, ANS, Max; char s [1005]; CIN> T; while (t --) {scanf ("% d", & N, & M); for (I = 0; I MAX) s [I] = 'C', max =
the network file sharing based on San, and the file access efficiency is high.
Good security
Access control for switch ports can be achieved through the zooning function of the fiber switch. Secure isolation at the LUN level through the Seastor disk array lun masking. File share access control is realized through software.
When the data is in a regular state of access, the data is stored in the SII 1000 fibre disk array system and can be accessed dir
the same method, the IDs of the modules with the same Tabid in the generated sew. EMS default dnn.
Of course, there is another way of thinking to achieve it. The general idea is similar to implementing banner ads indexing and searching. See below.
The customer needs text in the banner module, and the script should also be indexed to be searchable.
Banner is used to put advertisements on the website. The hyperlink URL of the advertisement bar that the customer wants to search on the search resul
fairly easy to add the shield icon to most UI elements:
ButtonsThis is very easy. A simple sendmessage call will do:SendMessage(GetDlgItem(hWnd, IDOK), BCM_SETSHIELD, 0, TRUE);Or you can use the new macro that essential does the same thing:Button_SetElevationRequiredState(hwndButton, fRequired);Unfortunately you cannot mark a button element in a dialog resource to include the shield icon. You'll have to write code in your wm_initdialog handler to take care of it.
Syslink/hyperlinkLayout an i
SAR was originally an internal tool, which can be downloaded at http://pagesperso-orange.fr/sebastien.godard/download.html.
1 InstallationTar zxvf xxx.tar.gz
./Configure
Make
Make install
2. Use Pidstat 2 5 // Displays the CPU usage of all active processes 5 times every 2 seconds. Pidstat - P 3132 2 5 // The CPU usage of processes whose PID is 3132 is displayed 5 times
Sar was originally an internal tool.
Sar was originally an internal tool, which can be downloaded at http://pagesperso-orange.fr/sebastien.godard/download.html.
1 installation
Tar zxvf xxx.tar.gz
./Configure
Make
Make install
2. use
Pidstat 2 5
// The CPU usage of all active processes is displayed 5 times every 2 seconds
Pidstat-p 3132 2 5
// The CPU usage of processes with a PID of 3132 is displayed 5 time
JSONSystem.Web.Script.Serialization.JavaScriptSerializer Scriptserializer =new System.Web.Script.Serialization.JavaScriptSerializer ();var jsonstr = scriptserializer.serialize (new {JSON =jsstr,navhtml=nav}); //Put two parameters into JsonstrContext. Response.Write (JSONSTR); Return to PageThe returned jsonstr,navhtml section is deleted, thus it can be seen that the "JSON" is followed by a string, so in the foreground data.json.ds[1].cou_id, can not be displayed, So we're going to turn the JSON
Sar was originally an internal tool, which can be downloaded at http://pagesperso-orange.fr/sebastien.godard/download.html.
1 Installation
Tar zxvf xxx.tar.gz
./Configure
Make
Make install
2. Use
Pidstat 2 5
// The CPU usage of all active processes is displayed 5 times every 2 seconds
Pidstat-p 3132 2 5
// The CPU usage of processes with a PID of 3132 is displayed 5 times every 2 seconds.
Pidstat-p
, managed, and like targeted activities. 2. Strong interest ListIn the 1920s, Edward strong of Stanford University Edward Strong A list of people's interests, reflecting specific career preferences. Strong believes that interest can bring something that we do not see in talent or achievement. These are the things people want to do and the things that make them happy.Today, Strong's list of interests (strong interesting Inventory, SII) includes people
(enable cpu1) 13. check the resources obtained by the process. cat/proc/3213/status14: group the cpu (default group:/) instance (create/cpusets cpu group) mkdir/cpusets grep cpu/proc/filesystems vim/etc/fstab mount-t cpuset nodev/cpusets/mount-a ls/cpusets /..... cpus ..... mem .... tasks... echo 1>/cpusets/cpus (allocate cpu to/cpusets) echo 0>/cpusets/mems (allocate mem to/cpusets) echo 3132>/cpusets/tasks (process number
c#2013101301
Here are two simple ways to demonstrate:
1. Use the shift character.
Cases:
byte[] bytes = new byte[2]{0x31,0x32};
Short U16;
U16 = (short) ((Bytes[0] Come to the result:
hex:3132
dec:12594
2. Use cast, 2nd byte *256
byte[] bytes = new byte[2]{0x31,0x32};
Short U16;
U16 = (short) (short) bytes[0] * 256 + (short) bytes[1];//There must be a cast in the front, because the middle 256 defaults to type int
button1. Text = U16. ToSt
Oracle's estimate based on statistics. For example, the Mytables table has 320,000 rows, the minimum value for the primary key myID is 1, and the maximum value is 409654, consider the following SQL statement: Select * from Mytables where myid>=1; The two seemingly similar SQL statements to the SELECT * from Mytables where myid>=400000, for Oracle, have a huge difference. Because the former FF is 100%, and the latter FF may be only 1%. If its CF is larger than the actual number of blocks, Oracle
]
col 7: [7] 6f 0a 1e 0d
Col 8:[19] 32 30 31 31 2 2d 3a 3132 3a
Col 3a 9: [2] C1
col: [5] 4e
col 11: [D 7] 6f 0a 1e 0d
bindmp:00 2a 0c 15 20 24 22
The real data content looks like this:
tab 0, row 0, @0x1da4
tl:7 fb:--h-fl--lb:0x0 cc:12 Col 0:*null* Col 1: [5] 4c 49 44
Col 2: [1] 4e
col 3:*null*
Col 4: [1] 4e
col 5: [1] 4e
Col 6: [3]
col 7: [7] 6f 0a 1e 0d
Col 8:[19] 32 30
estimate based on statistics. For example, the Mytables table has 320,000 rows, the minimum value for the primary key myID is 1, and the maximum value is 409654, consider the following SQL statement:
Select * from mytables where myid>=1; 和 Select * from mytables where myid>=400000
These two seemingly similar SQL statements, for Oracle, there is a huge difference. Because the former FF is 100%, and the latter FF may be only 1%. If its CF is larger than the actual number of blocks, Oracle may c
The content source of this page is from Internet, which doesn't represent Alibaba Cloud's opinion;
products and services mentioned on that page don't have any relationship with Alibaba Cloud. If the
content of the page makes you feel confusing, please write us an email, we will handle the problem
within 5 days after receiving your email.
If you find any instances of plagiarism from the community, please send an email to:
info-contact@alibabacloud.com
and provide relevant evidence. A staff member will contact you within 5 working days.